:100000000C9455070C94A8090C949C070C949C071D
:100010000C949C070C949C070C949C070C949C07D4
:100020000C949C070C949C070C94C6260C949A275D
:100030000C949A1D0C949C070C949C070C949C07A0
:100040000C949C070C949C070C949C070C949C07A4
:100050000C949C070C94001E0C949C070C949C0719
:100060000C949C070C949C070C949C070C949C0784
:100070000C949C070C949C070C949C070C949C0774
:100080000C949C070C949C070C949C070C949C0764
:100090000C949C070C949C070C949C070C949C0754
:1000A0000C949C070C949C070C949C0701E301E0C2
:1000B000014F024F02E002E30001E301E0015002C0
:1000C0005002E002E30001E30115021574FF02E3B0
:1000D00074FF010602060110021001070207012841
:1000E000022874FF01130213010C020C011102110A
:1000F000010A020A012C022C01E00119021902E096
:100100000001E30115021502E301060206011002D7
:1001100010010702070128022874FF74FF010C0276
:100120000C01130213010602060112021201110250
:100130001101090209010C020C010A020A012C0238
:100140002C0138023801040204010F020F010F02D2
:100150000F012802280001E30115021574FF02E3D4
:1001600074FF0106020601100210010702070128B0
:1001700002280001E0010402040106020602E00078
:1001800001E00119021902E00001E0010602060285
:10019000E000636D640128004143012800750A01F5
:1001A0002B022B010C020C01110211012B022B015D
:1001B000280228012B022B012B022B012B022B01E1
:1001C0000C020C01110211012B022B012802280044
:1001D000750A012B022B0112021201170217012BC3
:1001E000022B01280228012B022B012B022B012BB1
:1001F000022B011D021D01150215012B022B0128E6
:10020000022800750A012B022B01120212011302AF
:1002100013012B022B01280228012B022B012B0298
:100220002B012B022B011D021D01150215012B02B2
:100230002B01280228006970636F6E666967202FA2
:10024000616C6C00747300750A01270227010602B5
:1002500006012B022B012B022B01040204012B02AD
:100260002B00011B021B00750A01E0011702170198
:100270001902190128022802E0007777772E73759A
:1002800070706F72742E7865726F782E636F6D0167
:100290002800617061657A40676F746F636F732EB9
:1002A000636F6D0061646D696E012B313131310115
:1002B000280001E3012B022B02E3002E001E001F89
:1002C000002000210022002B4514001A0009001311
:1002D000000A00284004001500160017000700E17E
:1002E000001D001B00060019000500010001005060
:1002F000004F002A00DD5C0100010029613500008B
:100300003046002D00270026002500240023003160
:100310000033001C0018000F000D00280012000C14
:1003200000080011000B00350038003700360010BF
:10033000000E0001000100510052002C00280001B5
:100340000001004E004B00DE5C4C002E001E001F22
:10035000002000210022002B4514001A000800157F
:10036000001700284004001600070009000A00E1F9
:10037000001D001B0006001900050001004A0029AD
:100380000046000030DD5C2B451E001F00200021D0
:100390000022002D00270026002500240023003124
:1003A00000130012000C0018001C00280033000F7E
:1003B000000E000D000B003500380037003600102D
:1003C00000110001004D004A004C00DE5C28002DA9
:1003D000001F001F001F001F001F002E001E001F17
:1003E000002000210022002B0034003600370013CB
:1003F000001C00296104001200080018000C00E134
:1004000000330014000D000E001B002B451E001FC2
:10041000002000210022002B451E001F002000218B
:100420000022002D00270026002500240023002D97
:10043000000F00150006000A000900380016001120
:100440000017000B00070028401D0019001A0010BB
:100450000005002D001F001F001F001F001F002DA2
:10046000001F001F001F001F001F0035000C300D73
:10047000300E3001000100010001000330023001A4
:10048000000F3001000630010001000100010001F1
:100490000001000130010001000100005C010001C9
:1004A0000001000100005C2B45010001000100017A
:1004B000000100010030002F0001000100010001D7
:1004C000000A301030010001000100010001000BA2
:1004D00030520001000100010001004F00510050A6
:1004E000000100005C010001000100010001002D7D
:1004F000000100010001000100010035001E001F85
:100500000020002100220025001E0003301E001ED6
:10051000001E0025001E001E001E001E001E0025DD
:10052000001E001E001E001E001E002961E200E3E6
:10053000001E001E0035002B4501000100010001D6
:100540000001002D002700260025002400230000C4
:100550000056002300220021000000000057002068
:10056000001F001E000000000000003700270027C9
:10057000000000340001004F00500001004C002D2D
:10058000000100010001000100010045003A003BAC
:10059000003C003D003E0001002000200020002023
:1005A00000200001000100520001000100010029AB
:1005B00061E200E3000357DD5C2A002B451E001FAB
:1005C000002000210022002B451E001F00200021DA
:1005D000002200440043004200410040003F00016F
:1005E00000010001000100010001000100520001B2
:1005F000000100010001004F005100500034005282
:10060000002C002D00270026002500240023002DAB
:10061000001F001F001F001F001F0000000000003F
:1006200000000000000000000000000000000000CA
:1006300000000000000000000000000000000000BA
:1006400000000000000000000000000000000000AA
:10065000000000000000000000000000000000009A
:100BB00000000000000000000000000100DA5CDB23
:100BC0005CC15CC45CC35C0100DB5C01001D5C1E9D
:100BD0005C135C01001E001E000100010001000109
:100BE0000001000100DA5C010001000100010001C8
:100BF00000010001000100010001000100010001ED
:100C0000000100005C005CC75CC85CC55CC65C01A0
:100C100000015CDC5CDA5CDB5C0A5C010001000169
:100C200000010001000100010001000100010001BC
:100C300000010001000100010001000100010001AC
:100C4000000100010001000100010000000000009F
:100C50000000002A2B280000000000000000000017
:100C600000000000000029000000002C1E3420219C
:100C70002224342627252E362D3738271E1F2021E3
:100C800022232425263333362E37381F0405060742
:100C900008090A0B0C0D0E0F10111213141516175C
:100CA00018191A1B1C1D2F3130232D35040506077A
:100CB00008090A0B0C0D0E0F10111213141516173C
:100CC00018191A1B1C1D2F3130354C000000000074
:100CD0000000000000000000000000000000000014
:100CE0000000000000000000000000000101010100
:100CF00001010001010101000000000000000000EE
:100D000000000000000100010001010101010101DA
:100D100001010101010101010101010101010101C3
:100D200001010101010100000001010000000000BB
:100D300000000000000000000000000000000000B3
:100D40000000000000000101010100040330000068
:100D50000012034D0061006E00750066006F0072A6
:100D6000006D000000160343004800200062006F81
:100D70000078004D006F0064007300000004030958
:100D80000409025400030100A0FA09040000010351
:100D90000101000921110100012240000705810322
:100DA00008000A09040100010301020009211101E0
:100DB0000001224D000705820308000A0904020011
:100DC000010300000009211101000122360007057E
:100DD000830308000A1201100100000008EDFE6004
:100DE0003001000102030105010980A101850216FD
:100DF00001002603001A81002A83007510950181E5
:100E000000C0050C0901A1018503160100269C0202
:100E10001A01002A9C02751095018100C005010984
:100E200002A1010901A100050919012905150025E3
:100E3000019505750181029501750381010501097F
:100E40003009311581257F9502750881060938150D
:100E500081257F950175088106050C0A38021581E8
:100E6000257F950175088106C0C005010906A1010D
:100E7000050719E029E7150025019508750181028C
:100E80009501750881010508190129059505750168
:100E900091029501750391010507190029FF1500BD
:100EA00026FF00950675088100C011241FBECFEFF4
:100EB000DAE0DEBFCDBF04B603FE27C08091580242
:100EC00090915902A0915A02B0915B028730904BE9
:100ED000A740B04BD1F410925802109259021092D0
:100EE0005A0210925B0214BE84B7877F84BF0FB68C
:100EF000F894A895809160008861809360001092BA
:100F000060000FBEE0E0F8E3099511E0A0E0B1E079
:100F1000E4E2F4E502C005900D92A039B107D9F7DB
:100F200022E0A0E9B1E001C01D92A835B207E1F7C7
:100F30000E94F3230C94B0290C9400000C943A0BFB
:100F400080912B028B6080932B02ABE6B1E061E0D5
:100F500070E08D91E82FE295EF70F0E041A18F7085
:100F60009B0101C0220F8A95EAF7922F9095942356
:100F700091A382A1822B82A381E0A137B80749F710
:100F8000A5E6B1E061E070E08D91E82FE295EF70A9
:100F9000F0E041A18F709B0101C0220F8A95EAF712
:100FA000922F9095942391A382A1822B82A381E01A
:100FB000AB36B80749F7559A209AE0E9F1E0ADE978
:100FC000B1E08CE991E011921D928E179F07D9F73D
:100FD0000C94D60D3F924F925F926F927F928F92B8
:100FE0009F92AF92BF92CF92DF92EF92FF920F93B8
:100FF0001F93CF93DF9300D000D0CDB7DEB78091A1
:1010000000018111B0C086E090E09A838983098154
:101010001A8103561E4F8BE6E82E81E0F82E6801F8
:10102000AA24A394B12C8824839424E0922ED60180
:101030006D906D01FD011292FC83EB83D7018D91C0
:101040007D01E82FE295EF70F0E091A18F70B5017E
:1010500001C0660F8A95EAF7892F862B81A382A1AA
:10106000762E7094872182A3B0EABA95F1F745E60F
:1010700051E090E080E0DA015D90AD01252D2295F0
:101080002F7030E0D90190963C90AB81BC814C90A0
:10109000352D3F70D50102C0AA0FBB1F3A95E2F76C
:1010A0009D01232109F062C02A2D082E01C0220FC4
:1010B0000A94EAF72429AB81BC812C9301968630EF
:1010C0009105C9F681A1782271A282A1682B62A341
:1010D0008C91681659F08092A9010E94CA1D9093C4
:1010E000AB018093AA018BB189258BB9B1E7EB16CF
:1010F000B1E0FB0609F09BCF8091A9018823E1F0C4
:101100008091AA019091AB010E94D61D0697A0F094
:10111000E981FA81E057FE4FFA83E98380E0D80144
:101120009D918D01E981FA819193FA83E9838F5F23
:101130008630A9F71092A90181E00F900F900F90CF
:101140000F90DF91CF911F910F91FF90EF90DF9063
:10115000CF90BF90AF909F908F907F906F905F9057
:101160004F903F9008951A82198251CF20E0A2CF6C
:10117000CF93DF9380910001D0E0C0E0882311F08D
:10118000C6E0D0E00E940D0A009789F4C057DE4FF8
:1011900030E020E0F901E255FE4F408149932F5F96
:1011A0003F4F26303105B1F7DF91CF91089581E0AF
:1011B00090E0FACFCF930E94EA07C82F0E94B808A8
:1011C000892BE1F05D9880919C018F5F80939C0159
:1011D000863078F080910001F0E0E0E0882311F0A3
:1011E000E6E0F0E0E057FE4F86E090E011920197D4
:1011F000E9F70E94D80D8C2FCF9108955D9A109237
:101200009C01F7CF0E94EA0780910001E6E0F0E040
:10121000882311F0F0E0E0E0E057FE4F90E080E03E
:101220002191DC01A255BE4F2C9301968630910589
:10123000B9F70895E82FF0E0E057FE4F8081089558
:101240000895E8EDF0E08081806180838AE18A95ED
:10125000F1F700C08091D900817008958EE090E090
:101260000E947A2991E0811101C090E090930001E1
:101270000E942109882321F00E949B0978940895F7
:101280000E94C11D0E949F09F9CF0E94A0070E94E1
:101290000209FDCF0E942E090E942109811102C07E
:1012A0000E9445090895509A08955098589A0895B3
:1012B000589A08950E945509489BFECF80E88A9568
:1012C000F1F708950E94550998E080E029B1880F50
:1012D0002170822B20E82A95F1F725E02A95F1F775
:1012E0000000915099F708950F931F93CF93082F03
:1012F0000E945309C8E010E0C15020F4CF911F9123
:101300000F910895C8010C2E02C0959587950A94F7
:10131000E2F780FF06C00E94580980E88A95F1F73D
:10132000EBCF5898FACF0E945309589880E88A95D5
:10133000F1F70C9458090E9453090C9458090E9423
:101340005509E89AE9E6F0E080818C7F8083089572
:101350001F920F920FB60F921124EF92FF921F93DC
:101360002F933F934F935F936F937F938F939F93AD
:10137000AF93BF93CF93DF93EF93FF930E949309B3
:10138000D0E0C0E010E0CE0182559E4F7C01FC0110
:1013900080810E9474090E949309F7018081180FCF
:1013A0002196C630D10579F7812F0E9474090E94D9
:1013B0009309F0E8FA95F1F780E48A95F1F70E9435
:1013C00062098093AD010E949309D091AD010E9402
:1013D0006209C82F0E9493090E9455098091AC01AF
:1013E000DC17C9F081608093AC01FF91EF91DF9130
:1013F000CF91BF91AF919F918F917F916F915F91AD
:101400004F913F912F911F91FF90EF900F900FBE42
:101410000F901F9018958E7FE6CFEF92FF921F934B
:10142000CF93DF93F8940E945309589825E02A95AA
:10143000F1F700000E9455090E94580930E83A95DA
:10144000F1F789B1182F117080FF09C0789481E0FD
:1014500090E0DF91CF911F91FF90EF9008950E944F
:101460005A09D0E0C0E00E946209FE01E255FE4F39
:101470007F0180830E945A09F7018081180F21960D
:10148000C630D10581F70E946209C82F0E945A090F
:101490001C13DCCF8091AD010E9474090E945A098F
:1014A0008091AD010E9474090E945A090E9453095B
:1014B0000E945809789490E080E0CBCF0C94390BCF
:1014C000FC018081813021F489E891E00C944D1A6F
:1014D000823019F480E891E0F9CF83E791E0F6CF0C
:1014E000FC018081813021F486E591E00C944D1A55
:1014F000823019F481E091E0F9CF86EC90E0F6CFEC
:10150000FC018081813021F489EB90E00C944D1A2C
:10151000823019F48CEA90E0F9CF0895FC018081C3
:10152000813031F488E30E940D1388E30C94E813B2
:1015300081E30E940D1381E3F9CFCF93DF93EC0198
:101540000E94031DBE0190E080E0DF91CF910C94DA
:10155000D31ADC016131A0F4E62FF0E0EE54F64D31
:101560000C94602912968C91129781116DC012967D
:101570008C911297882339F084EA92E00E946D0DD5
:1015800090E080E0089512968C911297882319F0CC
:1015900082E992E0F3CF12968C911297882319F08A
:1015A0008AE792E0EBCF12968C91129781114FC08F
:1015B00015968C911597982F907F12962C91222337
:1015C00041F0992311F080FFDBCF83E00E94351BAF
:1015D000D7CF992311F080FF3DC083E00E94561BB6
:1015E000CFCF12968C911297811137C012968C91A1
:1015F0001297882319F084E492E0C0CF12968C9160
:101600001297882319F086E392E0B8CF12968C9156
:101610001297811125C012968C911297811123C0C7
:1016200012968C911297811121C012968C91882369
:1016300009F4A6CF88E991E0A1CF12968C9181118F
:101640009FCF82E991E09ACF82EB92E0089587E6FE
:1016500092E0089582E692E0089587E492E008958A
:1016600083E092E0089580ED91E008958DE991E0A6
:10167000089508950895CF93FB018C3D2CE59207C2
:1016800051F158F48A3D2CE59207B1F08B3D9C4511
:10169000E1F0C1E08C2FCF9108958E3D2CE59207AB
:1016A00061F1F8F0803E9C45A1F7C28180E1CC2336
:1016B00079F10E94351B07C0C28181E090E0CC2304
:1016C00049F30E949D0AC0E0E5CFC28182E090E02C
:1016D000CC2301F3F6CFC281CC23E1F284E090E089
:1016E000F0CFC28183E0CC2359F00E94351B40E14A
:1016F00064E083E00E94C40DE6CFC28184E0F3CFB2
:101700000E94561B40E164E083E00E94C40DC2CFFA
:101710000E94561BBFCF81E008950C943B0B0E94A2
:10172000DD162FEF84E39CE0215080409040E1F7EC
:1017300000C0000087E797E79093010880930008B6
:101740000C94241E0F931F93CF93DF938C01FC0105
:10175000C081D181CE010E94D11BBE010E94E20D49
:10176000EC01B8010E94EA10B801CE010E948D0B75
:10177000882309F459C0B801CE010E942E11882394
:1017800009F452C0B801CE010E943D10882309F42B
:101790004BC0C531FCE5DF0709F427C1B0F4C13007
:1017A000ECE5DE0709F446C008F056C0C115DC457B
:1017B000B1F181E08093B9018093BA01C801DF9152
:1017C000CF911F910F910C948B0BC53DECE5DE077B
:1017D00009F4F0C0B8F4C33D8CE5D80709F4AEC0F5
:1017E000C43DDC4531F7F8018281882309F4CDC07E
:1017F0001092BA010E94CA1D9093B8018093B7015C
:1018000080E2A9C0C83DFCE5DF07F1F0C93DDC4539
:1018100081F6F8018281882339F082E01AC0F8014C
:10182000828181110E948F0B80E0DF91CF911F9107
:101830000F910895F80182818823B1F380912B02E2
:10184000816080932B02F0CFF8018281882361F3BD
:1018500080E00E948E24E8CFF8018281882309F479
:10186000ADCF0E94F01C811102C00E94D61C0E94C4
:10187000081D90E090934A0280934902FE01E350D4
:10188000FC45809149028160E231F10538F4ED5365
:10189000F64D0C9460298091490282608093490240
:1018A000809149020E940C1D0E94DD16BDCF8091DF
:1018B00049028460F3CF809149028860EFCF809124
:1018C00049028061EBCF809149028062E7CF80912D
:1018D00049028064E3CF809149028068DFCF809124
:1018E00049028C60DBCF809149028E7FD7CF8091F7
:1018F00049028D7FD3CF809149028B7FCFCF8091DA
:101900004902877FCBCF809149028F7EC7CF8091DC
:1019100049028F7DC3CF809149028F7BBFCF8091D9
:1019200049028F77BBCF80914902837FB7CF9091D7
:101930004902892F97FB87F98058B0CFF80182813F
:10194000882361F01092B9010E94CA1D9093B601DC
:101950008093B50182E00E94371466CF8091B9016F
:1019600081110FC08091B5019091B6010E94D61DE2
:101970008639910530F486E20E940D1386E20E94BA
:10198000E81382E00E943E144FCF8091BA0181118A
:101990000FC08091B7019091B8010E94D61D863981
:1019A000910530F487E20E940D1387E20E94E8134C
:1019B00080E2E8CFF801828181111ACF8091BA01CB
:1019C0008111F6CF8091B7019091B8010E94D61D88
:1019D0008639910568F780E20E943E1488E20E94F1
:1019E0000D1388E20E94E8131FCF0E94971CF80194
:1019F0009281992381F08A7A91E009F490E09093A2
:101A0000B401811106C089E20E94201C0E94641C5E
:101A10000BCF85E3F9CF8091B401811104C089E235
:101A20000E94271CF3CF85E3FBCFCF9390E0FC010E
:101A3000E55BF34FC4918553934FFC018491882358
:101A400069F081EE0E940D138C2F0E940D138C2FD4
:101A50000E94E81381EECF910C94E8138C2F0E9422
:101A60000D138C2FF8CFFF920F931F93CF93DF931B
:101A70008C01F62EF8018491882349F1E801219622
:101A8000813049F4FE011491812F0E940D13812FA2
:101A90000E94E81306C0823089F4FE0184910E94FE
:101AA0000D138E010F5F1F4F8F2D815018F3EFE93B
:101AB000FFE03197F1F700C00000F7CF833019F451
:101AC000FE018491E5CF0E94150DE801EACFDF9178
:101AD000CF911F910F91FF90089560E00C94330D0A
:101AE0008F929F92AF92BF92CF92DF92EF92FF922E
:101AF0000F931F936B017C0181E090E0A0E0B0E0C8
:101B00004C015D0104C0880C991CAA1CBB1C4A95A1
:101B1000D2F7B501A4014C015D0104C0880C991CE9
:101B2000AA1CBB1C2A95D2F7482959296A297B2966
:101B300004C0880F991FAA1FBB1F0A95D2F78A01FC
:101B40009B010C211D212E213F210417150726077B
:101B5000370789F48C299D29AE29BF29BC01CD0105
:101B60001F910F91FF90EF90DF90CF90BF90AF90BB
:101B70009F908F90089580959095A095B0958C2119
:101B80009D21AE21BF21EACF0F93382F262F6091E0
:101B90001602709117028091180290911902042F79
:101BA000432F0E94700D0F910C940F1B0C945E0A32
:101BB0000E9488110C949E0708950C94DC0D0C94DF
:101BC000DD0D0895972F70E026E0929F600D711D46
:101BD0001124FB0198E4899FE00DF11D1124EE0F03
:101BE000FF1FE554FD4F859194910895FC01EE0F80
:101BF000FF1FE55BF24F859194910895CF93DF939A
:101C00000E94E20D0E949E0FEC01811520E59207D3
:101C100008F042C0811530E4930708F007C1883E00
:101C2000910528F5803E910508F09BC0883A910502
:101C300088F4853A910508F08AC08130910509F44D
:101C400090C0009709F48DC0049708F08AC0D0E0D6
:101C5000C0E087C08D3B910508F487C0805C910986
:101C6000C03CD105A0F30E94F60DEC017AC08115AD
:101C7000904250F4C11581E0D80708F072C0C03F0F
:101C8000D10528F3D0656DC0C11590E3D90708F0E0
:101C9000C3C0CE019F70E7CF811525E5920758F5A7
:101CA000811534E5930708F0F0C0811542E59407EB
:101CB00050F4C11581E5D80708F4BBC0DC2FCC2750
:101CC000C16FD06A4EC0982F969596959E0123704D
:101CD0003327C115D34508F0C9C0C1E0D0E002C028
:101CE000CC0FDD1F2A95E2F720E2929FC00111245C
:101CF000C82BD92BB9C0C11589E5D80780F4C11507
:101D000098E5D90708F0C6C0C11526E5D20708F046
:101D10009ECFDC2FCC27CC27DF71D06222C0CE0132
:101D2000C1153AE5D30708F4BAC090568115904220
:101D300008F08DCF8D2F8F710E94191090E0982F91
:101D4000882788279F719C012C2BE901E6CF853AD3
:101D5000910509F4AEC0863A910509F0ADC0C2E81C
:101D6000D0E4CE01DF91CF910895883A910509F42E
:101D7000A6C0893A910509F4A5C08A3A910509F4EB
:101D8000A4C08B3A910509F4A3C08C3A910509F4DB
:101D9000A2C08B3B910509F4A1C08C3B910509F4CD
:101DA000A0C08D3A910509F49FC0803B910509F4CC
:101DB0009EC08E3A910509F49DC08F3A910509F4B1
:101DC0009CC0813B910509F49BC0823B910509F4BD
:101DD0009AC0833B910509F499C0843B910509F4AD
:101DE00098C0853B910509F497C0863B910509F49D
:101DF00096C0873B910509F495C0883B910509F48D
:101E000094C0893B910509F493C08A3B910509F47C
:101E100092C0C0E0D4E4A5CFCE019927D3FF03C080
:101E2000EC01D86C9ECFEC01D06C9BCFDF70D06AF8
:101E300098CFCE01E4E096958795EA95E1F7837017
:101E40002C2F26952695237090E2299F900111242E
:101E5000382B8C2F8370C1E0D0E002C0CC0FDD1F87
:101E60008A95E2F7C22BD32BDC687BCFC1E0D0E0B0
:101E700002C0CC0FDD1F2A95E2F730E2939FC0012C
:101E80001124C82BD92BDA686CCFD82FCC27C46F7C
:101E9000D06A67CFDC2FCC27C06FD06A62CF34E026
:101EA000969587953A95E1F78F70CF70C06ED82FD1
:101EB000BECFC1E8D0E455CFC3E8D0E452CFC2EEE4
:101EC000D4E44FCFC9EED4E44CCFCAEED4E449CF2A
:101ED000C5EBD4E446CFC6EBD4E443CFC3EBD4E4A4
:101EE00040CFC4EBD4E43DCFC7EBD4E43ACFCCEC45
:101EF000D4E437CFCDECD4E434CFC3E8D5E431CF4C
:101F0000CAE8D5E42ECFC2E9D5E42BCFC4E9D5E4A5
:101F100028CFC1E2D6E425CFC3E2D6E422CFC4E283
:101F2000D6E41FCFC5E2D6E41CCFC6E2D6E419CF73
:101F3000C7E2D6E416CFCAE2D6E413CF82389105C1
:101F400049F1B0F48133910509F462C048F4893253
:101F5000910509F456C08A32910509F460C00895CC
:101F60008533910509F446C08933910599F00895A8
:101F7000833E910531F138F4803E910591F0823E27
:101F80009105B1F00895863E910521F1873E9105B6
:101F900051F10895209149022370D9F080EE90E02C
:101FA00008952091490220FF14C089E390E008952C
:101FB0002091490222FF0DC024FD09C083EE90E06C
:101FC00008952091490222FD31C024FF02C090E013
:101FD00080E008952091490223FFFBCF24FDF7CF35
:101FE00087EE90E008952091490223FFEECF86EE20
:101FF00090E008952091490225FFEBCF89E290E01F
:1020000008952091490225FFE4CF85E390E00895EB
:102010002091490226FFDDCF8AE290E008952091C9
:10202000490226FFD6CF81E390E0089582EE90E04A
:1020300008959091490292FF06C0282F28712830F8
:1020400069F4877F846093FF06C0282F28712831A8
:1020500061F4877E846194FD877E0895282F247122
:10206000243089F78B7F8860EECF282F24712431AC
:1020700091F78B7E8861EFCF08950F931F93CF93D5
:102080008C01FB018281811106C0C1E08C2FCF91B0
:102090001F910F910895C091C801C11125C006314B
:1020A0001C4599F70E943C1081E08093C8010E9472
:1020B000CA1D9093C7018093C6011092BB01109274
:1020C000BD011092BC011092BF011092BE0110928E
:1020D000C1011092C0011092C3011092C20110926E
:1020E000C5011092C401D2CF8091C6019091C70161
:1020F0000E94D61D8C32914040F68091BB01E82FA2
:10210000F0E0EE0FFF1FE454FE4F118300838F5F5A
:102110008093BB01C0E0BACFCF93DF93EC0181E0A5
:102120008F878F810E949A1C88850E94AD1C0E9417
:10213000641CEA81FB81309739F06A897B89CE0182
:102140000696DF91CF910994DF91CF910895EF9298
:10215000FF920F931F93CF93DF93EC01888581113A
:1021600032C0EB80FC8087E5F81A24E12E9DC00187
:102170002F9D900D1124DC01AF5FBE4F1496ED91A1
:10218000FC911597309731F052966D917C91895F53
:102190009E4F099584E18E9D80018F9D100D112425
:1021A0000F5F1E4FF80187810E94A01CF8018085F7
:1021B0000E94B31C0E94641C18821F821986109210
:1021C000CA011092C901DF91CF911F910F91FF9029
:1021D000EF900895DF92EF92FF920F931F93CF93AA
:1021E000DF937C01FB018281882391F08091510172
:1021F0008F3F71F0C1E0D1E010E000E0DD24D39426
:1022000080915101082E000C990B8017910744F41E
:10221000DF91CF911F910F91FF90EF90DF90089584
:102220008E818823B9F089859A858E159F0539F4AA
:102230008091C9019091CA018E159F0559F0DD86E4
:102240008F85811103C0CE010E948C10CE010696AD
:102250000E94A7100F5F1F4F6496D2CFEF92FF929C
:102260000F931F93CF93DF937C0197558F3F910579
:1022700009F0D8F520915101022E000C330B2817DC
:10228000390714F480935101FB01228134E1389F16
:102290008001399F100D1124E801CF5FDE4F2E879A
:1022A00092818E81992349F1FA86E9868F5F8E8328
:1022B0000E94CA1D9C878B870E94D31C8F830E941B
:1022C000971C88870E94AA1C9885892B8887E8819B
:1022D000F981309731F06A897B89C801895F9E4F07
:1022E0000995F092CA01E092C90181E0DF91CF9196
:1022F0001F910F91FF90EF9008958823B1F38F8580
:10230000882399F3C801895F9E4F0E94A710EDCFE3
:10231000EF92FF920F931F93CF93DF938091510120
:1023200010E004E18F3FC1F5DF91CF911F910F9134
:10233000FF90EF900895029FF001039FF00D11248C
:10234000EF5FFE4FE088F188E114F10419F486E9AB
:10235000E82EF12C029FE001039FD00D1124CF5FE6
:10236000DE4F8E818823B9F08B859C850E94D61D17
:10237000E816F90680F4109F700111248F858111F1
:1023800005C0C7018F5F9E4F0E948C10C701895FF7
:102390009E4F0E94A7101F5F212F30E080915101B6
:1023A000082E000C990B821793072CF6BDCF909343
:1023B000D0018093CF010895E091CF01F091D00139
:1023C000309721F00190F081E02D099480E008958C
:1023D000E091CF01F091D001309721F00280F3819C
:1023E000E02D09940895E091CF01F091D00130974C
:1023F00021F00480F581E02D099408952091CD010C
:102400003091CE012817390771F09093CE01809357
:10241000CD01E091CF01F091D001309721F00680FD
:10242000F781E02D099408952091CB013091CC01E2
:102430002817390771F09093CC018093CB01E0917C
:10244000CF01F091D001309721F00084F185E02D8B
:10245000099408950C944A0981E008950E94C11DD1
:102460000E94A0070C94351EBF92CF92DF92EF928C
:10247000FF920F931F93CF93DF93CDB7DEB72A97C9
:102480000FB6F894DEBF0FBECDBF0E94DA080E94DF
:102490002C12882309F471C082EDC82E81E0D82E59
:1024A00010E000E0B02E802F0E941A09E82EF601FD
:1024B000F1906F01F81609F45AC080912B0281FD4A
:1024C0000E94200990E080E0FE242F2D30E0482F6C
:1024D000B901082E02C0759567950A94E2F760FF6E
:1024E00041C08E83BF8281E090E06C0102C0CC0CC1
:1024F000DD1C4A95E2F72E2D30E02C213D21232BC7
:1025000009F480E088870E94CA1D8160782F9A872D
:1025100089874E815F8168858A850E94DE12F80175
:10252000EE52FE4F80818C2580830E94C31F0E9443
:10253000DC119091D101891789F10E94DC118093FF
:10254000D1012A960FB6F894DEBF0FBECDBFDF9142
:10255000CF911F910F91FF90EF90DF90CF90BF90A0
:102560000C94DF0D01968630910509F0B0CF0F5F16
:102570001F4F0C30110509F095CF8FEF89838A83A7
:102580001B820E94CA1D8160782F9D838C834981A4
:102590005A816B818D810E94DE12C7CF2A960FB6B9
:1025A000F894DEBF0FBECDBFDF91CF911F910F9189
:1025B000FF90EF90DF90CF90BF900895CF93DF937F
:1025C000CDB7DEB72B970FB6F894DEBF0FBECDBFE9
:1025D0004F83588769877A878B871E821D8285E0A3
:1025E000FE013796DE01119601900D928A95E1F772
:1025F00049815A816B817C818D819E812B960FB69A
:10260000F894DEBF0FBECDBFDF91CF910C94B3190C
:10261000FC01808191810C94131CCF93C82F8823D7
:1026200009F4D4C08238C1F40E94DC1181FDCEC00F
:1026300089E30E94201C0E94641C2FEF81EE94E02D
:10264000215080409040E1F700C0000089E30E94E3
:10265000271CCF910C94641C8338A1F40E94DC11D8
:1026600080FDB4C083E50E94201C0E94641C2FEFF3
:1026700081EE94E0215080409040E1F700C00000DE
:1026800083E5E5CF8438A1F40E94DC1182FD9EC071
:1026900087E40E94201C0E94641C2FEF81EE94E0CE
:1026A000215080409040E1F700C0000087E4CFCF88
:1026B0008CEF8C0F813A48F48C2F0E94C521811138
:1026C00085C08C2F0E94201CC4CF80E28C0F8830E4
:1026D00048F4C77081E001C0880FCA95EAF70E94EC
:1026E0009A1CB7CF8BE58C0F833068F481E890E0BB
:1026F000C53A31F083E890E0C63A11F482E890E000
:10270000CF910C94FE1188E58C0F853108F05EC0E6
:1027100082EE90E0C83A09F456C089EE90E0C93ADA
:1027200009F451C08AEE90E0CA3A09F44CC085EB36
:1027300090E0CB3A09F447C086EB90E0CC3A09F43C
:1027400042C083EB90E0CB3BF1F184EB90E0CC3BDB
:10275000D1F187EB90E0CD3AB1F18CEC90E0C03B49
:1027600091F18DEC90E0CE3A71F183E891E0CF3AAF
:1027700051F18AE891E0C13B31F182E991E0C23B3D
:1027800011F184E991E0C33BF1F081E292E0C43BB6
:10279000D1F083E292E0C53BB1F084E292E0C63B27
:1027A00091F085E292E0C73B71F086E292E0C83B8F
:1027B00051F087E292E0C93B31F090E080E0CA3B03
:1027C00011F48AE292E0CF910C941412CF91089503
:1027D000882309F44BC0823871F40E94DC1181FF18
:1027E00045C089E30E94201C0E94641C89E30E946A
:1027F000271C0C94641C833859F40E94DC1180FF60
:1028000035C083E50E94201C0E94641C83E5EFCF45
:10281000843859F40E94DC1182FF28C087E40E94AA
:10282000201C0E94641C87E4E2CF9CEF980F913A31
:10283000F0F290E2980F983050F4877091E001C068
:10284000990F8A95EAF7892F0E94A01CD2CF9BE5A9
:10285000980F933020F490E080E00C94FE11885A99
:10286000853120F490E080E00C94141208958823C0
:1028700021F00E949A1C0C94641C0895882321F076
:102880000E94A01C0C94641C08958F929F92AF929A
:10289000BF92CF92DF92EF92FF920F931F93CF934D
:1028A000DF937C01D62FC72FFC01058102950F70A5
:1028B000128111110E94BA1C0E945D1CC82E88232F
:1028C00071F01123B1F080E28D0F883090F082E03A
:1028D0000E94471C0E945D1C91E0C82EC926DC2E78
:1028E000D2949FE0D922ED2DF0E0EB52F64D0C94FE
:1028F0006029C12CF4CF0C2F0F70C07F11F002950E
:10290000007F1123A9F0002359F080E28D0F883059
:1029100010F0D11109C0802F0E949A1C0E94641CE3
:102920008D2F0E940D1314C0802F0E94AD1CF6CF76
:102930008D2F0E94E813002359F080E28D0F88301C
:1029400010F0D11133C0802F0E94A01C0E94641C83
:1029500098E0D91639F0D91648F086E08D0D8F70C1
:10296000823020F40E94DC110E94DF0DCC2009F49B
:10297000D9C10E943A1C80FDD5C1F70112820E9484
:10298000341C0E94351BC7010E949F160E94341CF4
:10299000DF91CF911F910F91FF90EF90DF90CF903B
:1029A000BF90AF909F908F900C94561B802F0E94E9
:1029B000B31CCCCFFC2FFF70BF2EC07FC03219F0EC
:1029C000B29480EFB822DD2369F0D13049F11123B0
:1029D00091F1002351F1F701858180FFA1CF8F7024
:1029E000858323C0112381F0011106C00E94D31CEE
:1029F0008B290E943714ACCF0130C1F70E94D31C41
:102A00008B290E94CD1CA4CF011106C00E94D01CAE
:102A10008B2D0E943E149CCF013009F499CFF6CF44
:102A2000112329F0063008F093CF8B2DE2CF05302B
:102A300008F08ECFEDCF002359F38D2F0E94E813BD
:102A400087CF8C2F86958695837069F0813009F049
:102A50007FCF8D2F9C2F9370111102C090E080E0EA
:102A60000E94141275CF8D2F9C2F9370111102C0EC
:102A700090E080E00E94FE116BCF112309F1D53F59
:102A800099F0D63FB9F0D43F49F480914302909138
:102A90004402816090934402809343028D2F0E94F0
:102AA000D11E0E94B81F54CF8091430290914402DE
:102AB0008260F0CF80914302909144028460EACF1B
:102AC000D53F89F0D63FA9F0D43F49F48091430225
:102AD000909144028E7F90934402809343028D2F05
:102AE0000E94391FDECF80914302909144028D7F76
:102AF000F2CF80914302909144028B7FECCF8C2FD8
:102B0000837009F047C0111123CF2D2F22952695F0
:102B10002770220F220F6D2F6F70862E912CB12CF3
:102B2000A12C022E04C0880C991CAA1CBB1C0A9460
:102B3000D2F760E070E0CB01D4FF0FC06FE070E02F
:102B400080E090E004C0660F771F881F991F2A95C8
:102B5000D2F76095709580959095C695C695C3708F
:102B6000C23051F080F4682979298A299B29C13023
:102B700071F00E94E71AECCE682979298A299B29ED
:102B80000E94F91AE5CE0E94E71AC501B4010E941D
:102B9000D51ADECE8695112311F08C2F81708823F3
:102BA00009F4D6CE2D2F229526952770220F220FBD
:102BB0006D2F6F70862E912CB12CA12C022E04C08B
:102BC000880C991CAA1CBB1C0A94D2F760E070E028
:102BD000CB01D4FF0FC06FE070E080E090E004C054
:102BE000660F771F881F991F2A95D2F760957095F9
:102BF00080959095C695C695C370C23051F080F40B
:102C0000682979298A299B29C13071F00E94AC1B5F
:102C10009FCE682979298A299B290E94BE1B98CEBC
:102C20000E94AC1BC501B4010E949A1B91CEE0E248
:102C3000ED0FE53108F04DC0F0E0EB51F64D0C948E
:102C40006029DF708C2F8F71112321F00E94351BBA
:102C50008D2FCFCE0E94561B8D2FDBCE112341F03E
:102C6000053008F075CE8C2F8F710E94791B70CEC5
:102C7000063008F06DCEF7CF8C2F8F71112339F00D
:102C80000E94351B65CE8C2F8F711123C9F30E94D2
:102C9000561B5ECE112329F08C2F8F710E94201BB2
:102CA00057CE0E941B1B54CE112349F0CF718C2F9D
:102CB0000E94351B63E08C2F0E943E1C49CE81E0B0
:102CC0000E94471C023008F443CE82E00E94471C59
:102CD0003FCE112329F0011123CE8C2F8F71D0CF3D
:102CE000002369F0D93309F0A8CEFFEF27EE83E087
:102CF000F15020408040E1F700C000009ECE8C2FB4
:102D00008F71C5CF4C2F4F706D2FC7010E94A90A3C
:102D10000E944D1A1DCE4C2F4F706D2FC7010E947F
:102D2000E10D16CEDF91CF911F910F91FF90EF90A3
:102D3000DF90CF90BF90AF909F908F9008950F93AA
:102D40001F93CF93DF93EC018B819C81892B29F01A
:102D50008881998189238F3F29F4DF91CF911F9139
:102D60000F910895CE010E94A20B8823B1F36881D0
:102D700079818A810E941D1C8C010E94D01B0E94B7
:102D8000D21AB801CE01DF91CF911F910F910C940F
:102D900045140E94BA1C0E94CA1C0E942E1C0E944C
:102DA000641C0E944D200E94B81F90E080E00E94A9
:102DB000FE1190E080E00C9414120E94A71C0C9469
:102DC000C9160E94131CE92FE295EF70E250EE3015
:102DD00070F4F0E0E650F64D0C946029803F19F055
:102DE00020F4803E20F481E00895843FE1F380E008
:102DF0000895803EC0F3813FD1F7F5CF93FB88273C
:102E000080F90895CF93DF9300D000D00F92CDB713
:102E1000DEB70F900F900F900F900F90DF91CF9132
:102E20000895CF93DF9300D000D000D0CDB7DEB7A8
:102E300026960FB6F894DEBF0FBECDBFDF91CF91BF
:102E400008951F93CF93DF93C091DE0116E0809128
:102E5000DF018C1304C0DF91CF911F910895D0E062
:102E60001C9FF0011D9FF00D1124E052FE4F408188
:102E7000518162817381848195810E94111721960D
:102E8000C770E5CF4091100250911102609112027B
:102E90007091130280911402909115020C941117F5
:102EA0002091DE019091DF0156E0291302C080E0FD
:102EB000089530E0529FF001539FF00D1124E0522D
:102EC000FE4F7181761306C07081781303C0728142
:102ED000741304C02F5F3F4F2770E7CF81E0089540
:102EE0001F93CF93DF9380911502807FC1F480916F
:102EF00012028823A1F08091DE01C091DF01609170
:102F00001002709111024091130250911402D62FB9
:102F1000D723DA01A095B09516E0C81304C0DF915D
:102F2000CF911F91089590E04115510511F0DF3FB9
:102F300031F401968770F1CF2A0F3B1F17C0189FFD
:102F4000F001199FF00D1124E052FE4F218127134B
:102F5000F0CF20812613EDCF22812111EACF2381EA
:102F600034812417350740F3241B350B26393105EE
:102F700000F7209115022F7020612093150226E0A2
:102F8000289FF001299FF00D1124EB51FE4F808105
:102F90008F708061808380E192E00E949F16DF91B4
:102FA000CF911F910C9421179F92AF92BF92CF9215
:102FB000DF92EF92FF920F931F93CF93DF93CDB7E2
:102FC000DEB761970FB6F894DEBF0FBECDBF8C01A0
:102FD00085E0F801DE011D9601900D928A95E1F7DA
:102FE000D801DC901196EC9011971296CC90129724
:102FF0008091130290911402009709F492C12091DC
:10300000100230911102422F43234F3F09F489C12E
:103010001396AD90BC9090901202992009F422C1B1
:10302000A816B906E0F1F501E81BF90BCF01FF2462
:10303000F3948639910508F0F12C80911502982FB0
:10304000907FFF2009F4C7C091118EC0FC2C3E1167
:103050002BC02D1129C0C11027C08F7080618093B3
:1030600015020E94421780E192E00E949F16809113
:103070001502D80115968C938F2D61960FB6F89492
:10308000DEBF0FBECDBFDF91CF911F910F91FF909B
:10309000EF90DF90CF90BF90AF909F900895809574
:1030A00090958A0D9B1DC3CFA114B10429F08E2DDC
:1030B0008D218F3F09F054C180E080FF16C04C2D58
:1030C0006E2D8D2D0E945017882379F080E192E0BB
:1030D0000E949F1686E0E0E1F2E0DF011D928A95F2
:1030E000E9F70E944217F12CC7CFAB2829F08E2DAB
:1030F0008D218F3F09F031C180E0B82FB170AB2E28
:1031000080FF29C04C2D6E2D8D2D0E945017B82E9A
:10311000811121C0DD86EE868D859E850E94131C5F
:10312000292F22952F70223050F0243078F49F7090
:1031300051F0F8019581907F31F4FB2C9DCF9F7069
:1031400011F08823D1F3805E8830B8F3C8010E9463
:103150009F16BA2CF2CFCC2009F48ECF80911502A5
:10316000816080931502BFCF3E1106C02D1104C0AF
:10317000D801CC2009F49CC0DD86EE868D859E8525
:103180000E94E116882319F1CC2009F180911502E3
:10319000803270F0209110023091110238872F8315
:1031A0001986BB86AA868C87CE0107960E949F1639
:1031B00086E0F801A0E1B2E001900D928A95E1F776
:1031C0000E9470170E944217FF24F39455CFC80144
:1031D0000E949F16F9CF911115C07A2DB98AA88A3D
:1031E0004D2D5E2D6C2D89890E94021780E192E0A1
:1031F0000E949F1686E0E0E1F2E0DF011D928A95D1
:10320000E9F763C03E1112C02D1110C0C1100EC0ED
:10321000F8018583C8010E949F16E0E1F2E086E094
:10322000DF011D928A95E9F7F92C26CFDD86EE861F
:103230008D859E850E94E116882349F2CC2039F2C3
:1032400080911502803208F4B3CF209110023091A2
:1032500011023A8329831B82BD82AC828E83CE0108
:103260000196A4CFA816B90698F1F501E81BF90B51
:10327000CF01F12C8639910508F049C0FC2CCC20F7
:1032800009F4A5CF3E1132C02D1130C08091150236
:1032900080FD23C0982F907F01F1D80115968C9363
:1032A0001597903F39F0982F907F905F8F70892B02
:1032B00015968C93C8010E949F1686E0F801A0E144
:1032C000B2E001900D928A95E1F70E944217D4CEA8
:1032D000809590958A0D9B1DCCCF86E0F801A0E1EA
:1032E000B2E001900D928A95E1F7C6CEDD86EE86BA
:1032F0008D859E850E94E11681115ACF809115021D
:10330000816080931502C8010E949F16B5CE7A2D68
:10331000B98AA88A4D2D5E2D6C2D89890E940217CD
:1033200069CFCC2009F453CFDD86EE868D859E854E
:103330000E94E116F82E882309F449CF86E0F801AF
:10334000A0E1B2E001900D928A95E1F780E192E070
:103350000E9408130E947017B8CF81E08C25CDCE53
:1033600081E08C25AACE1F93CF93DF93CDB7DEB734
:103370002C970FB6F894DEBF0FBECDBF4F83588792
:1033800069877A878B879C87CE0107960E94D4171E
:10339000882369F08A859B85892B39F04F81588570
:1033A000842F85238F3F09F071C016E05FC086E04F
:1033B000FE013796DE01119601900D928A95E1F794
:1033C0008A859B85892B89F388859F8189238F3FF7
:1033D00061F32091DF0130E0C901019687709927E0
:1033E0004091DE014817190671F40E94DD16109213
:1033F000DF011092DE0186E0E0E1F2E0DF011D92E4
:103400008A95E9F7D2CF96E0929FD001939FB00DB5
:103410001124A052BE4FFE01319601900D929A9553
:10342000E1F78093DF010E942117BFCF819FC00188
:10343000112480529E4F0E94D4178823E9F0E09116
:10344000DE011E9FF0011124E052FE4F40815181A8
:1034500062817381848195810E9411178091DE01C0
:1034600090E00196877099278093DE018091DE01BC
:103470009091DF018913DACF2C960FB6F894DEBF56
:103480000FBECDBFDF91CF911F91089569857A85D9
:103490008B859C850E94111788CFEF92FF920F9326
:1034A0001F93CF93DF938C01892B81F0F12CEE24B5
:1034B000E394E8012196F8018491843770F4843014
:1034C00008F05FC08130B1F08230A1F1DF91CF917F
:1034D0001F910F91FF90EF900895853709F44CC02C
:1034E00008F43DC09CE7980F903780F78F770E94D3
:1034F000E81349C00E5F1F4FFE01849190E2980FC0
:10350000983060F48770FE2D01C0FF0F8A95EAF7AE
:103510008F2F0E94BD1C0E94641C02C00E940D13CC
:103520008F2D815030F2EFE9FFE03197F1F700C0C5
:103530000000F7CF0E5F1F4FFE01849190E2980FBD
:10354000983050F48770FE2D01C0FF0F8A95EAF77E
:103550008F2F0E94C31CDFCF0E94E813E1CF0E5FC4
:103560001F4FFE01C491C150D8F28FE99FE001972F
:10357000F1F700C00000F7CF0E5F1F4FFE01F4907F
:10358000CFCF0E940D138E01CBCF08950E94C51A94
:1035900060931A0270931B0280931C0290931D0289
:1035A0000C94C91608950C94C61A0F931F9300919A
:1035B0001A0210911B0220911C0230911D02602BF7
:1035C000712B822B932B1F910F910C94C61A0F9382
:1035D0001F9300911A0210911B0220911C0230913E
:1035E0001D0260237123822393231F910F910C945A
:1035F000C61A0F931F9300911A0210911B0220917B
:103600001C0230911D0260277127822793271F918A
:103610000F910C94C61A0C94C51A0C940B1B0E94A3
:103620000D1B6093160270931702809318029093FB
:1036300019020C94C91660E070E0CB010C940F1BCA
:103640000F931F9341E050E060E070E08A019B011E
:1036500004C0000F111F221F331F8A95D2F7C90122
:10366000B8011F910F910C940F1B0F931F9341E012
:1036700050E060E070E004C0440F551F661F771FE4
:103680008A95D2F78091160290911702A0911802A4
:10369000B09119028A019B01082B192B2A2B3B2B75
:1036A000C901B8011F910F910C940F1B0F931F9329
:1036B00041E050E060E070E004C0440F551F661F19
:1036C000771F8A95D2F7CB01BA01609570958095E6
:1036D00090950091160210911702209118023091D6
:1036E000190260237123822393231F910F910C945D
:1036F0000F1B0F931F9341E050E060E070E004C0A7
:10370000440F551F661F771F8A95D2F780911602C6
:1037100090911702A0911802B09119028A019B01A1
:10372000082719272A273B27C901B8011F910F91A4
:103730000C940F1B0F931F93009116021091170208
:103740002091180230911902602B712B822B932B40
:103750001F910F910C940F1B0F931F930091160252
:1037600010911702209118023091190260237123E1
:10377000822393231F910F910C940F1B0F931F9380
:10378000009116021091170220911802309119022F
:1037900060277127822793271F910F910C940F1B8D
:1037A0000895BF92CF92DF92EF92FF920F931F93F3
:1037B000CF93DF938C01C0901602D0901702E09057
:1037C0001802F090190280911A0290911B02A091A8
:1037D0001C02B0911D02C82AD92AEA2AFB2ACFE18D
:1037E000D0E0BC2ED701C6010C2E04C0B695A7951B
:1037F000979587950A94D2F780FD0EC0219788F798
:10380000B12C8B2DDF91CF911F910F91FF90EF90F5
:10381000DF90CF90BF900895B8018C2F0E94FE0DCD
:10382000019761F3EECFCF93DF93EC010E94D11BA0
:10383000BE01DF91CF910C94FE0DCB010C94131CB3
:10384000682F80915201909153010C94451D682F6F
:1038500080915201909153010C94471D8091520127
:10386000909153010C94491D80911E028595859578
:103870008595089580911E028770089598E0899F2C
:1038800090011124622B60931E020C94351B9091C1
:103890001E028095892380931E02282F277061F4D1
:1038A000282F082E000C330B9217130629F085954C
:1038B000859585950C94561B089590911E029770DE
:1038C00081E009F480E00895E0915201F091530104
:1038D00080912A028083E0915201F091530180810E
:1038E00090912902892B8083E0915201F09153013C
:1038F000808190912802892B808390911F029923C7
:1039000081F0E0915201F09153018081892B8083F5
:1039100080915201909153010E94111D81111092CA
:103920001F0280915201909153010C94E8118091F3
:103930002A02089590912A02892B80932A020895E1
:10394000809590912A02982390932A0208951092CC
:103950002A02089580912902089590912902892BC5
:10396000809329020895809590912902982390933D
:103970002902089510922902089590912802892B16
:10398000809328020895809590912802982390931F
:103990002802089510922802089580931F02089526
:1039A00010921F02089580911F0208956DEE7EEF20
:1039B00090E080E00E949A2960E082E090E00E941E
:1039C000882960E083E090E00E94882960E084E03C
:1039D00090E00E94882960E085E090E00C948829BE
:1039E00090E080E00E94822921E08D3E9E4F09F008
:1039F00020E0822F089582E090E00C947A2983E001
:103A000090E00C947A29682F83E090E00C94882948
:103A100084E090E00C947A29682F84E090E00C9484
:103A20008829FC0131969C01285F3F4F80E09191ED
:103A300091118F5FE217F307D1F708959C01FC0104
:103A400032969FEF80E04191461751F09F3F19F465
:103A5000411101C0982F8F5F8630A9F79F3F09F46D
:103A60000895290F311D97FD3A95F9016283089554
:103A7000FC01329608962191261303C0DF011197AD
:103A80001C92E817F907B9F708950C941E1D0C94C1
:103A9000381DFC0111821282138214821582168253
:103AA0001782089580914F02843039F110922C02D0
:103AB00088E190E020E40FB6F894A8958093600028
:103AC0000FBE2093600080E00E94DF0D83B7817FEE
:103AD000846083BF83B7816083BF7894889583B700
:103AE0008E7F83BF0FB6F894A8958091600088619F
:103AF00080936000109260000FBE089508950895AD
:103B0000CF930E947E1D0E94DA080E947F1DC0E0B4
:103B10008C2F0E941A09811105C0CF5FCC30C1F7EC
:103B2000CF91089581E0FCCF0E94DD160E94DC1148
:103B30000C94DF0D1F921FB61F9211248F939F9339
:103B4000AF93BF9380912C02811113C080914502E5
:103B500090914602A0914702B09148024196A11D62
:103B6000B11D8093450290934602A0934702B09303
:103B70004802BF91AF919F918F911F901FBE1F90E0
:103B8000189582E084BD93E095BD9AEF97BD809330
:103B90006E0008952FB7F8948091450290914602E7
:103BA000A0914702B09148022FBF0895CF92DF92B3
:103BB000EF92FF920F931F932FB7F8944091450215
:103BC0005091460260914702709148022FBF6A01EE
:103BD0007B01EE24FF248C0130E020E0C016D106EA
:103BE000E206F30650F0481B590BCA011F910F91D2
:103BF000FF90EF90DF90CF90089541505109F3CF9F
:103C000078941F921FB61F9211248F939F93AF93A6
:103C1000BF938091450290914602A0914702B091D6
:103C200048020196A11DB11D809345029093460262
:103C3000A0934702B0934802BF91AF919F918F919B
:103C40001F901FBE1F90189587E797E79093010874
:103C50008093000888E19AE00FB6F894A8958093C5
:103C600060000FBE90936000FFCF0E94F01C811196
:103C700002C00E94D61C0E94FB1C80932B020E9453
:103C8000081D90E090934A02809349020E94FF1C15
:103C9000682F70E090E080E00C94D31A80912F029E
:103CA00080FF12C06091570185E0689FB001112428
:103CB000759567957595679560387105A8F56115D7
:103CC0007105A1F1862F089581FF09C06091570108
:103CD00085E0689FB001112475956795EDCF6091DF
:103CE000570182FD0AC0809130028823D1F0909163
:103CF000560160915701891728F085E0689FB0014F
:103D00001124DACF869FB001112485E0869F9001AF
:103D1000879F300D1124692F70E0C9010E944C2942
:103D2000CBCF65E070E0CECF8FE7089581E00895B6
:103D300080912F0280FF0CC06091550170E0759555
:103D40006795759567956115710549F1862F0895F9
:103D500081FF06C06091550170E075956795F3CFBE
:103D60006091550182FD0BC0909130029923A1F022
:103D70006091540180915501961738F0682F70E0DA
:103D80006038710500F38FE70895899FC001112401
:103D900070E00E944C29F4CF61E070E0D7CF81E061
:103DA0000895803F31F40E944E1E81958093330226
:103DB0000895813F19F40E944E1EF8CF823F31F4DE
:103DC0000E944E1E8195809332020895833F19F41C
:103DD0000E944E1EF8CF893F29F40E94981E8093BE
:103DE000340208958A3F21F40E94981E8195F7CFEE
:103DF0008B3F31F40E94981E81958093350208957F
:103E00008C3F19F40E94981EF8CF843F31F48091C2
:103E100031028160809331020895853F21F48091C1
:103E200031028260F7CF863F21F4809131028460B5
:103E3000F1CF873F21F4809131028860EBCF883F3A
:103E400021F4809131028061E5CF8D3F31F4809182
:103E50002F02816080932F0208958E3F21F480917C
:103E60002F028260F7CF8F3FB9F780912F028460D5
:103E7000F1CF90913202803F41F48091330287FD6F
